:100000000C9449000C943B010C9464010C948D01F8
:100010000C9466000C9466000C9466000C946600C8
:100020000C9466000C9466000C9466000C94DE013F
:100030000C9466000C947D000C9466000C94660091
:100040000C9466000C9466000C9466000C94660098
:100050000C94660050756C736520656E65726769F7
:1000600065733A2000566361702072656D61696E38
:10007000696E673A200046495245210A0053706F65
:10008000742057656C646572205265736574210A2B
:10009000000011241FBECFE5D8E0DEBFCDBF10E0C9
:1000A000A0E6B0E0EAEDFBE002C005900D92A439B5
:1000B000B107D9F710E0A4E9B0E001C01D92AB3D53
:1000C000B107E1F70E94B3030C94EB050C94000018
:1000D000FC01849105C05D9BFECF8CB93196849163
:1000E0008823C9F70895FC0104C05D9BFECF8CB93D
:1000F000319680818823C9F708951F920F920FB619
:100100000F9211248F939F93EF93FF939CB1809153
:1001100095008823F9F49CB99A3031F09D3021F094
:10012000809194008F3361F481E080939500E09199
:100130009400F0E0E556FF4F1082109294000AC040
:1001400080919400E82FF0E0E556FF4F90838F5F99
:1001500080939400FF91EF919F918F910F900FBE2C
:100160000F901F901895882359F02FE088E190E0B8
:100170000FB6F894A89581BD0FBE21BDA89508952E
:10018000A89588E10FB6F89481BD11BC0FBE089503
:10019000909196009923E1F0913009F041C08823B5
:1001A00021F080919A008F5F03C080919A00815066
:1001B00080939A0080919A0087FF05C080919A00F1
:1001C0008F5F80939A0080919A0010929A00089510
:1001D00020918F0030919000882319F02F5F3F4FBE
:1001E00002C0215030403093900020938F008091C6
:1001F0008F00909190000A9730F48AE090E09093FD
:10020000900080938F0080918F00909190008F5587
:10021000914030F08EE591E09093900080938F00B4
:100220000895882329F0662359F0633029F408C023
:10023000662311F0633021F480919900815003C04E
:10024000809199008F5F809399008091990084300C
:1002500029F481E00E94C8001092990080919900D1
:100260008C3F29F480E00E94C80010929900089504
:100270008091960008951F920F920FB60F9211244D
:100280002F933F934F935F936F937F938F939F939E
:10029000AF93BF93EF93FF9360B3669566956370DA
:1002A00080E00E941101FF91EF91BF91AF919F916A
:1002B0008F917F916F915F914F913F912F910F900F
:1002C0000FBE0F901F9018951F920F920FB60F92AE
:1002D00011242F933F934F935F936F937F938F934B
:1002E0009F93AF93BF93EF93FF9360B3669566952B
:1002F000637081E00E941101FF91EF91BF91AF9176
:100300009F918F917F916F915F914F913F912F912D
:100310000F900FBE0F901F9018951F920F920FB65F
:100320000F9211242F933F934F935F936F937F937B
:100330008F939F93AF93BF93EF93FF938BB78F7D73
:100340008BBF8BB78F7D8BBF86B3482F447082FFE6
:100350000CC084B78F7B84BF20919800922F80E0DF
:1003600022B730E0282B392B06C084B7806484BFC5
:1003700012BE109298008AB78F7D8ABF8BB78062B9
:100380008BBF8BB780628BBF442339F080E0295B41
:100390003B4008F081E00E943801FF91EF91BF914E
:1003A000AF919F918F917F916F915F914F913F910D
:1003B0002F910F900FBE0F901F9018951F920F92C4
:1003C0000FB60F9211248F93809198008F5F8093C6
:1003D00098008F910F900FBE0F901F90189512BE2E
:1003E00085E083BF1CBE89B7816089BF8A98929AD5
:1003F0008B98939ABA98C29A85B7816085BF85B762
:100400008D7F85BF8BB780648BBF85B7846085BFC8
:1004100085B7877F85BF8BB780688BBF84B78F7B9D
:1004200084BF8BB780628BBF08950197F1F7089561
:10043000CF93DF93EC0105C086E69EE00E94150293
:1004400021972097C9F7DF91CF9108951F93182F17
:1004500005C080E791E00E94150211501123C9F7F1
:100460001F9108951F93182F05C084E290E00E9409
:10047000150211501123C9F71F9108951F93162FCC
:10048000909197008295880F880F807C9061982BBF
:1004900095BB82E390E00E94150285B31F70812B0B
:1004A00085BB82E390E00E941502AC9882E390E065
:1004B0000E941502AC9A82E390E00E9415021F91FF
:1004C00008951F93909197008295880F880F807CE4
:1004D0009063982B95BB82E390E00E941502AC9844
:1004E00082E390E00E94150213B3AD9882E390E09E
:1004F0000E941502812F8F701F9108950F931F93F3
:10050000182F80EF84BB82E390E00E941502812FB8
:100510000E946102082F812F0E9461020295007FD4
:10052000802B1F910F9108958FEF84BB80E29EE492
:100530000E94150280E063E00E943E0280E197E2A3
:100540000E94150280E063E00E943E0284EF91E089
:100550000E94150280E063E00E943E0280E062E0BB
:100560000E943E0208950F931F93182F062F629545
:100570006F700E943E02812F602F0E943E021F91E9
:100580000F91089580E061E00E94B30280E395E757
:100590000E94150208950E94940280E068E20E9481
:1005A000B30280E068E00E94B3020E94C20280E0D1
:1005B00066E00E94B30280E06CE00E94B3020895FE
:1005C000CF93DF93EC0108C06A3019F480E060EC4F
:1005D00001C081E00E94B30221966A9121966623B0
:1005E00099F7DF91CF9108950F931F93CF93DF93E6
:1005F000082F282F392FE90104C0219681E00E949D
:10060000B302CE01801B182F68816623B1F705C0A5
:1006100081E060E20E94B3021F5F1830C8F3DF91EF
:10062000CF911F910F910895962F682F6295660FB5
:10063000660F607C690F605880E00E94B3020895E5
:1006400087B987ED86B9349BFECF24B130E045B140
:10065000942F80E0282B392BC90108950E94200394
:10066000A0E0B0E0BC01CD0128E934E040E050E07A
:100670000E947A0523E030E040E050E00E94AD05A2
:100680008AE056954795379527958A95D1F7C90100
:100690000895DF92EF92FF920F931F937C01D62E65
:1006A0008A01CA0160E670E00E944205F801D48226
:1006B000C7016AE070E00E949905805D8383C701ED
:1006C0006AE070E00E9499059B01CB016AE070E04E
:1006D0000E949905805D8283C9016AE070E00E94F2
:1006E0009905CB016AE070E00E949905805D8083E6
:1006F0001F910F91FF90EF90DF900895DF92EF929E
:10070000FF920F931F937C01D62E8A01CA0166E6E1
:1007100070E00E944205F801D482C7016AE070E0EF
:100720000E949905805D8383C7016AE070E00E94A2
:1007300099059B01CB016AE070E00E949905805DFC
:100740008183C9016AE070E00E949905CB016AE0EB
:1007500070E00E949905805D80831F910F91FF904A
:10076000EF90DF900895A2E2B0E0E9EBF3E00C94A3
:10077000CF0510BC8FE289B988E98AB98EE880BDBF
:100780008FB780688FBFB89AC098B998C19A8C9A71
:1007900094988D9A95988E9A96980E94CB028CE6A2
:1007A00090E00E94E0028DE790E00E94680084EFF4
:1007B00091E00E9418020E94C2020E94EF0100E034
:1007C00064E0A62EB12CAC0EBD1E5AE0652E712C35
:1007D0006C0E7D1E4FE0242E312C2C0E3D1E34E17C
:1007E000432E512C4C0E5D1E2CC0C02EDD24F60174
:1007F000EF56FF4FE0808E2D90E0A0E0B0E08F8FAD
:1008000098A3A9A3BAA3802F0E942003A1E0B0E07F
:10081000AC0FBD1FCA0EDB1E0196A0E0B0E0BC010C
:10082000CD012F8D38A149A15AA10E947A052AE055
:1008300096958795779567952A95D1F7F601608308
:100840000F5F033090F283E00E942E037C0184E06E
:100850000E942E038C0195989498969880918F0011
:10086000909190000817190708F4949A0196801740
:10087000910708F4969A80919600813091F1C70112
:1008800060E2A3010E947E0380918F00909190000E
:1008900060E2A1010E947E03C80160E2A2010E9401
:1008A0007E0380E060E00E941403C3010E94E00226
:1008B000898190E060E2A3010E9449038A8190E06F
:1008C00060E2A1010E947E038B8190E060E2A201C0
:1008D0000E947E0381E060E00E941403C3010E9435
:1008E000E00280918F0090919000801B910BFFEFB0
:1008F0008F3F9F070CF4BEC002970CF0BBC0C09A9C
:10090000B199BAC086E790E00E9468008981882387
:1009100019F0959A0E94320295988A810E942602C7
:1009200084E00E942E034C018B81882319F0959A54
:100930000E942602959881E090E00E94180284E0CF
:100940000E942E036C0160E2A5010E947E030E94BA
:10095000C20280E060E00E94140388E790E00E94F9
:10096000E00280E06AE00E941403C5010E94E002F8
:1009700085E690E00E946800C5010E94730083E84C
:1009800090E00E94730084E590E00E94680081E09E
:1009900060E00E94140385E890E00E94E002889CD9
:1009A0007001899CF00C989CF00C1124009FB00100
:1009B000019F700D109F700D11246E197F0980E04A
:1009C00090E02EE530E040E050E00E947A0520E122
:1009D00037E240E050E00E94AD05DA01C901B501FF
:1009E0004AE050E00E944905C5010E9473008DE86D
:1009F00090E00E94730081E067E00E941403C5014B
:100A00000E94E002CC9CC001CD9C900DDC9C900D1E
:100A10001124E81AF90AC701A0E0B0E08B8F9C8F7F
:100A2000AD8FBE8FBC01CD012EE530E040E050E03F
:100A30000E947A0520E137E240E050E00E94AD05D7
:100A4000DA01C901B5014AE050E00E944905C5013B
:100A50000E94730083E890E00E94730081E06BE0E5
:100A60000E941403C5010E94E002B19BFECF0E94C8
:100A7000C20202C0C098959885E090E00E941802DA
:100A800000E0B3CEFB01DC0101900D920020E1F704
:100A90000895FB019F01E8944230C4F04532B4F45C
:100AA0004A3029F497FB1EF4909581959F4F642F4F
:100AB00077270E949905805D8A330CF0895D8193C8
:100AC000CB010097A1F716F45DE251931082C901A2
:100AD0000C946A05DC01FC01672F71917723E1F723
:100AE000329704C07C916D9370836291AE17BF07FB
:100AF000C8F30895629FD001739FF001829FE00DBB
:100B0000F11D649FE00DF11D929FF00D839FF00D8C
:100B1000749FF00D659FF00D9927729FB00DE11D38
:100B2000F91F639FB00DE11DF91FBD01CF01112415
:100B30000895AA1BBB1B51E107C0AA1FBB1FA61724
:100B4000B70710F0A61BB70B881F991F5A95A9F776
:100B500080959095BC01CD010895A1E21A2EAA1BA3
:100B6000BB1BFD010DC0AA1FBB1FEE1FFF1FA2175D
:100B7000B307E407F50720F0A21BB30BE40BF50B5A
:100B8000661F771F881F991F1A9469F760957095E3
:100B9000809590959B01AC01BD01CF0108952F92E6
:100BA0003F924F925F926F927F928F929F92AF92FD
:100BB000BF92CF92DF92EF92FF920F931F93CF934A
:100BC000DF93CDB7DEB7CA1BDB0B0FB6F894DEBFE1
:0A0BD0000FBECDBF0994F894FFCFCB
:100BDA00202E2020200020202E20200053706F7409
:100BEA002057656C6465720056636170206C656697
:100BFA007420000A0050756C73204520002000788C
:040C0A0000C89696F2
:00000001FF
